Archive member included       because of file (symbol)

casllib.a(caslpro_event_handler.o)
                              casl_events.o (CASLpro_event_handler)
/prc-tools/H-i586-cygwin32/m68k-palmos/lib/libcrt.a(hooks.o)
                              /prc-tools/H-i586-cygwin32/m68k-palmos/lib/gcrt0.o (__do_bhook)
/prc-tools/H-i586-cygwin32/m68k-palmos/lib/libcrt.a(gdbstub.o)
                              /prc-tools/H-i586-cygwin32/m68k-palmos/lib/gcrt0.o (_GdbStartDebug)
/prc-tools/H-i586-cygwin32/m68k-palmos/lib/libcrt.a(multi_dreloc.o)
                              obwheel-sections.o (_GccLoadCodeAndRelocateData)
/prc-tools/H-i586-cygwin32/m68k-palmos/lib/libcrt.a(reloc_chain.o)
                              /prc-tools/H-i586-cygwin32/m68k-palmos/lib/libcrt.a(multi_dreloc.o) (_RelocateChain)
/prc-tools/H-i586-cygwin32/lib/gcc-lib/m68k-palmos/2.95.2-kgpd/libgcc.a(_ltdf2.o)
                              obwheel.o (__ltdf2)
/prc-tools/H-i586-cygwin32/lib/gcc-lib/m68k-palmos/2.95.2-kgpd/libgcc.a(_gtdf2.o)
                              obwheel.o (__gtdf2)
/prc-tools/H-i586-cygwin32/lib/gcc-lib/m68k-palmos/2.95.2-kgpd/libgcc.a(_eqdf2.o)
                              obwheel.o (__eqdf2)
/prc-tools/H-i586-cygwin32/lib/gcc-lib/m68k-palmos/2.95.2-kgpd/libgcc.a(_double.o)
                              obwheel.o (__adddf3)
/prc-tools/H-i586-cygwin32/lib/gcc-lib/m68k-palmos/2.95.2-kgpd/libgcc.a(fpgnulib.o)
                              caslprop.o (__floatsidf)
/prc-tools/H-i586-cygwin32/lib/gcc-lib/m68k-palmos/2.95.2-kgpd/libgcc.a(_fixunsdfsi.o)
                              caslprop.o (__fixunsdfsi)
/prc-tools/H-i586-cygwin32/lib/gcc-lib/m68k-palmos/2.95.2-kgpd/libgcc.a(_umodsi3.o)
                              casl_support_pilot.o (__umodsi3)
/prc-tools/H-i586-cygwin32/lib/gcc-lib/m68k-palmos/2.95.2-kgpd/libgcc.a(_nedf2.o)
                              casl_support_pilot.o (__nedf2)
/prc-tools/H-i586-cygwin32/lib/gcc-lib/m68k-palmos/2.95.2-kgpd/libgcc.a(_ledf2.o)
                              casl_support_pilot.o (__ledf2)
/prc-tools/H-i586-cygwin32/lib/gcc-lib/m68k-palmos/2.95.2-kgpd/libgcc.a(_gedf2.o)
                              casl_support_pilot.o (__gedf2)
/prc-tools/H-i586-cygwin32/lib/gcc-lib/m68k-palmos/2.95.2-kgpd/libgcc.a(_floatex.o)
                              /prc-tools/H-i586-cygwin32/lib/gcc-lib/m68k-palmos/2.95.2-kgpd/libgcc.a(_double.o) (_fpCCR)
/prc-tools/H-i586-cygwin32/lib/gcc-lib/m68k-palmos/2.95.2-kgpd/libgcc.a(_udivsi3.o)
                              /prc-tools/H-i586-cygwin32/lib/gcc-lib/m68k-palmos/2.95.2-kgpd/libgcc.a(_umodsi3.o) (__udivsi3)
/prc-tools/H-i586-cygwin32/lib/gcc-lib/m68k-palmos/2.95.2-kgpd/libgcc.a(_mulsi3.o)
                              /prc-tools/H-i586-cygwin32/lib/gcc-lib/m68k-palmos/2.95.2-kgpd/libgcc.a(_umodsi3.o) (__mulsi3)
/prc-tools/H-i586-cygwin32/m68k-palmos/lib/libg.a(bcopy.o)
                              pilotsock.o (bcopy)

Allocating common symbols
Common symbol       size              file

scratch_char_buf    0x190             casl_pilotmain.o
color_depth         0x4               casl_pilotmain.o
framergb            0x4               casl_pilotmain.o
errno               0x2               casl_pilotmain.o
platform_version    0x4               casl_pilotmain.o
fldhighliteforergb  0x4               casl_pilotmain.o
formbackrgb         0x4               casl_pilotmain.o
__casl_constants    0x2               obwheel.o
forergb             0x4               casl_pilotmain.o
gNetLibOpen         0x2               casl_pilotmain.o
AppINETString       0x20              casl_pilotmain.o
cur_xpen            0x2               casl_pilotmain.o
text_fore_index     0x4               casl_pilotmain.o
fldlinesrgb         0x4               casl_pilotmain.o
text_back_index     0x4               casl_pilotmain.o
AppServInfo         0x46              casl_pilotmain.o
selectedforergb     0x4               casl_pilotmain.o
formforergb         0x4               casl_pilotmain.o
AppHostInfo         0x238             casl_pilotmain.o
fldhighlitebackrgb  0x4               casl_pilotmain.o
sock_objs           0x14              casl_pilotmain.o
frame_fore_index    0x4               casl_pilotmain.o
fldcaretrgb         0x4               casl_pilotmain.o
frame_back_index    0x4               casl_pilotmain.o
backrgb             0x4               casl_pilotmain.o
selectedbackrgb     0x4               casl_pilotmain.o
generic_fore_index  0x4               casl_pilotmain.o
object_ptr          0x4               casl_pilotmain.o
inet_sock_objs      0x28              casl_pilotmain.o
fldtextrgb          0x4               casl_pilotmain.o
cur_ypen            0x2               casl_pilotmain.o
linger_structure    0x4               netfile.o
generic_back_index  0x4               casl_pilotmain.o
fldbackrgb          0x4               casl_pilotmain.o

Memory Configuration

Name             Origin             Length             Attributes
coderes          0x00000000         0x0000fde8
datares          0x00000000         0x00007fff
caslsuppres      0x00000000         0x00008000
caslnetwres      0x00000000         0x00008000
*default*        0x00000000         0xffffffff

Linker script and memory map


.text           0x00000000     0x69c0
 *(.text)
 .text          0x00000000       0xa0 /prc-tools/H-i586-cygwin32/m68k-palmos/lib/gcrt0.o
                0x00000000                start
 .text          0x000000a0     0x4d26 obwheel.o
                0x00000bd0                fxnpvD_cf_
                0x000031e0                fxneleveN_cf_
                0x00002d56                fxnminusyeaR_cf_
                0x000003c0                fxnnuL_cf_
                0x00000d16                fxnnumtodaY_cf_
                0x00004776                fxnsavepasS_cf_
                0x000035b8                fxnthirtY_cf_
                0x00003210                fxntwelevE_cf_
                0x000035ec                fxnthirtyonE_cf_
                0x000049dc                _pda_init_caslpro_app
                0x00003b16                fxnuS_cf_
                0x00004500                fxndefaulT_cf_
                0x00004722                fxncleaR_cf_
                0x000037a8                fxnbishoP_cf_
                0x0000486a                fxncheckiT_cf_
                0x0000351c                fxntwentyseveN_cf_
                0x00003090                fxnfouR_cf_
                0x0000337c                fxnnineteeN_cf_
                0x00002b10                fxnmaincalC_cf_
                0x000028c4                fxncalclmpfredC_cf_
                0x0000372a                fxnsettodaY_cf_
                0x00004170                fxnlaunchpT_cf_
                0x00004d84                _pda_shutdown_caslpro_app
                0x00000494                fxnposT_cf_
                0x0000263e                fxncalc2trI_cf_
                0x00002f40                fxnseP_cf_
                0x000000a0                _pda_dbcreator_id
                0x00002426                fxncalclmpyeaR_cf_
                0x0000042a                fxnprE_cf_
                0x00002ee0                fxnjuL_cf_
                0x000046f8                fxnseekpasS_cf_
                0x00003480                fxntwentyfouR_cf_
                0x0000104e                fxnnumfromtwO_cf_
                0x0000062e                fxndropstA_cf_
                0x0000344c                fxntwentythreE_cf_
                0x00002baa                fxnsetdateS_cf_
                0x00004192                fxnlmP_cf_
                0x00002e20                fxnmaR_cf_
                0x0000491c                fxnsubmiT_cf_
                0x00002fd0                fxndeC_cf_
                0x0000463a                fxnopendatabaseS_cf_
                0x000031b0                fxnteN_cf_
                0x00002cec                fxnplusyeaR_cf_
                0x00003150                fxneighT_cf_
                0x00000356                fxnproM_cf_
                0x00002fa0                fxnnoV_cf_
                0x00003060                fxnthreE_cf_
                0x00004992                fxnnexT_cf_
                0x000032e0                fxnsixteeN_cf_
                0x000046c0                fxnreadpasS_cf_
                0x00003244                fxnthirteeN_cf_
                0x000034b4                fxntwentyfivE_cf_
                0x00000c72                fxncalcbishoP_cf_
                0x00004680                fxnpasspositioN_cf_
                0x00002f70                fxnocT_cf_
                0x00002eb0                fxnjuN_cf_
                0x000049d0                shutdowN_cf_
                0x000033b0                fxntwentY_cf_
                0x000032ac                fxnfifteeN_cf_
                0x000030c0                fxnfivE_cf_
                0x000044ae                fxnabouT_cf_
                0x00000c7e                fxnbacK_cf_
                0x00003626                fxnsetdateiN_cf_
                0x00000c18                fxnclearbishoP_cf_
                0x0000141c                fxncalcmmdD_cf_
                0x0000011c                fxnlasT_cf_
                0x00003180                fxnninE_cf_
                0x00003120                fxnseveN_cf_
                0x00000ca4                fxnnumtodatE_cf_
                0x000049bc                startuP_cf_
                0x00001a0e                fxncalctri1_cf_
                0x000033e4                fxntwentyonE_cf_
                0x00004662                fxnclosedatabaseS_cf_
                0x00002e80                fxnmaY_cf_
                0x00002df0                fxnfeB_cf_
                0x000044d4                fxnbackabouT_cf_
                0x00002a16                fxndedC_cf_
                0x00002334                fxncalcedcyeaR_cf_
                0x000030f0                fxnsiX_cf_
                0x00003348                fxneighteeN_cf_
                0x00002512                fxncalc1trI_cf_
                0x0000291c                fxncalcuS_cf_
                0x00003584                fxntwentyninE_cf_
                0x00003e44                fxnedC_cf_
                0x00003314                fxnseventeeN_cf_
                0x00003550                fxntwentyeighT_cf_
                0x00002e50                fxnapR_cf_
                0x00002dc0                fxnjaN_cf_
                0x000007bc                fxndropefF_cf_
                0x00003418                fxntwentytwO_cf_
                0x00000a7a                fxndropdiL_cf_
                0x000047ea                fxncheckpasS_cf_
                0x0000282e                fxncalcedcfrlmP_cf_
                0x000034e8                fxntwentysiX_cf_
                0x00001e9c                fxncalctri2_cf_
                0x000026d2                fxncalcagE_cf_
                0x000037e8                fxndatE_cf_
                0x000010c0                fxnnumfroM_cf_
                0x00003278                fxnfourteeN_cf_
                0x00000948                fxndroppoS_cf_
                0x0000050c                fxndropcoN_cf_
                0x00002f10                fxnauG_cf_
                0x00003030                fxntwO_cf_
                0x00003000                fxnonE_cf_
 *fill*         0x00004dc6        0x2
 .text          0x00004dc8        0x4 obwheel-sections.o
                0x00004dc8                _GccRelocateData
 .text          0x00004dcc      0x6ac casl_pilotmain.o
                0x00005050                PilotMain
                0x000052a4                _dbfile_rec_compare
                0x00005434                _GccReleaseCode
                0x00005244                _pda_strcmp
                0x0000530e                sort_synced_databases
 .text          0x00005478      0x188 caslprop.o
                0x00005558                pda_visual_object_and_color_ptr
                0x00005508                _pda_object_geometry_ptr
                0x00005478                pda_visual_object_ptr
 .text          0x00005600      0x104 casl_support_pilot.o
                0x0000561a                _draw_bitmap
                0x00005600                _pda_hardware
 .text          0x00005704      0x144 casl_support.o
                0x0000574e                validate_property
 .text          0x00005848       0xf8 pilotsock.o
                0x00005872                OpenInetLib
 .text          0x00005940        0xa casllib.a(caslpro_event_handler.o)
                0x00005940                CASLpro_event_handler
 *fill*         0x0000594a        0x2
 .text          0x0000594c      0x110 /prc-tools/H-i586-cygwin32/m68k-palmos/lib/libcrt.a(hooks.o)
                0x00005a22                __do_dtors
                0x000059e8                __do_ctors
                0x0000594c                __do_bhook
                0x0000599a                __do_ehook
 .text          0x00005a5c       0x62 /prc-tools/H-i586-cygwin32/m68k-palmos/lib/libcrt.a(gdbstub.o)
                0x00005a5c                _GdbStartDebug
 *fill*         0x00005abe        0x2
 .text          0x00005ac0       0xac /prc-tools/H-i586-cygwin32/m68k-palmos/lib/libcrt.a(multi_dreloc.o)
                0x00005ac0                _GccLoadCodeAndRelocateData
 .text          0x00005b6c       0x26 /prc-tools/H-i586-cygwin32/m68k-palmos/lib/libcrt.a(reloc_chain.o)
                0x00005b6c                _RelocateChain
 *fill*         0x00005b92        0x2
 .text          0x00005b94       0x1c /prc-tools/H-i586-cygwin32/lib/gcc-lib/m68k-palmos/2.95.2-kgpd/libgcc.a(_ltdf2.o)
                0x00005b94                __ltdf2
 .text          0x00005bb0       0x1c /prc-tools/H-i586-cygwin32/lib/gcc-lib/m68k-palmos/2.95.2-kgpd/libgcc.a(_gtdf2.o)
                0x00005bb0                __gtdf2
 .text          0x00005bcc       0x1c /prc-tools/H-i586-cygwin32/lib/gcc-lib/m68k-palmos/2.95.2-kgpd/libgcc.a(_eqdf2.o)
                0x00005bcc                __eqdf2
 .text          0x00005be8      0xa08 /prc-tools/H-i586-cygwin32/lib/gcc-lib/m68k-palmos/2.95.2-kgpd/libgcc.a(_double.o)
                0x000064c6                __cmpdf2
                0x00005c5c                __adddf3
                0x0000645e                __negdf2
                0x000061c6                __divdf3
                0x0000600a                __muldf3
                0x00005c56                __subdf3
 .text          0x000065f0      0x1b2 /prc-tools/H-i586-cygwin32/lib/gcc-lib/m68k-palmos/2.95.2-kgpd/libgcc.a(fpgnulib.o)
                0x00006788                __fixsfsi
                0x000065f0                __floatsidf
                0x00006636                __extendsfdf2
                0x0000670a                __fixdfsi
                0x0000661e                __floatsisf
                0x0000668e                __truncdfsf2
 *fill*         0x000067a2        0x2
 .text          0x000067a4       0x62 /prc-tools/H-i586-cygwin32/lib/gcc-lib/m68k-palmos/2.95.2-kgpd/libgcc.a(_fixunsdfsi.o)
                0x000067a4                __fixunsdfsi
 *fill*         0x00006806        0x2
 .text          0x00006808       0x2a /prc-tools/H-i586-cygwin32/lib/gcc-lib/m68k-palmos/2.95.2-kgpd/libgcc.a(_umodsi3.o)
                0x00006808                __umodsi3
 *fill*         0x00006832        0x2
 .text          0x00006834       0x1c /prc-tools/H-i586-cygwin32/lib/gcc-lib/m68k-palmos/2.95.2-kgpd/libgcc.a(_nedf2.o)
                0x00006834                __nedf2
 .text          0x00006850       0x1c /prc-tools/H-i586-cygwin32/lib/gcc-lib/m68k-palmos/2.95.2-kgpd/libgcc.a(_ledf2.o)
                0x00006850                __ledf2
 .text          0x0000686c       0x1c /prc-tools/H-i586-cygwin32/lib/gcc-lib/m68k-palmos/2.95.2-kgpd/libgcc.a(_gedf2.o)
                0x0000686c                __gedf2
 .text          0x00006888       0x86 /prc-tools/H-i586-cygwin32/lib/gcc-lib/m68k-palmos/2.95.2-kgpd/libgcc.a(_floatex.o)
                0x0000689e                $_exception_handler
                0x00006888                __clear_sticky_bit
 *fill*         0x0000690e        0x2
 .text          0x00006910       0x5e /prc-tools/H-i586-cygwin32/lib/gcc-lib/m68k-palmos/2.95.2-kgpd/libgcc.a(_udivsi3.o)
                0x00006910                __udivsi3
 *fill*         0x0000696e        0x2
 .text          0x00006970       0x22 /prc-tools/H-i586-cygwin32/lib/gcc-lib/m68k-palmos/2.95.2-kgpd/libgcc.a(_mulsi3.o)
                0x00006970                __mulsi3
 *fill*         0x00006992        0x2
 .text          0x00006994       0x26 /prc-tools/H-i586-cygwin32/m68k-palmos/lib/libg.a(bcopy.o)
                0x00006994                bcopy
 *fill*         0x000069ba        0x2
                0x000069bc                .=ALIGN(0x4)
                0x000069bc                bhook_start=.
 *(bhook)
                0x000069bc                bhook_end=.
                0x000069bc                .=ALIGN(0x4)
                0x000069bc                ehook_start=.
 *(ehook)
 ehook          0x000069bc        0x4 obwheel-sections.o
                0x000069c0                ehook_end=.
                0x000069c0                .=ALIGN(0x4)
                0x000069c0                ctors_start=.
 *(.ctors)
                0x000069c0                ctors_end=.
                0x000069c0                .=ALIGN(0x4)
                0x000069c0                dtors_start=.
 *(.dtors)
                0x000069c0                dtors_end=.

.data           0x00000000     0x1cf4
                0x00000000                data_start=.
 *(.data)
 .data          0x00000000     0x1358 obwheel.o
                0x00000040                icoN_cv_
                0x0000006c                choosemontH_cv_
                0x00000002                _casl_status_vaR_cv_
                0x0000001c                errorcodE_cv_
                0x00000054                toP_cv_
                0x000001a0                numdtypE_cv_
                0x00000168                numtodaY_cv_
                0x00000144                dpstA_cv_
                0x00000014                bytesreaD_cv_
                0x00000050                sidE_cv_
                0x000001b8                chooseyeaR_cv_
                0x00000024                curdiR_cv_
                0x00000362                __casl_objects
                0x00000360                __num_casl_objects
                0x00000198                numtypE_cv_
                0x00000128                dppoS_cv_
                0x0000009c                choosedaY_cv_
                0x00000180                nummmdD_cv_
                0x0000002c                platforM_cv_
                0x000001bc                dbregobw_field_map
                0x00000044                larroW_cv_
                0x00000004                invokeR_cv_
                0x00000064                passstrinG_cv_
                0x000001b0                numyeaR_cv_
                0x00001354                __num_constant_bytes
                0x00000048                rarroW_cv_
                0x00000154                dpcoN_cv_
                0x00000000                _casl_loop_vaR_cv_
                0x00000038                _casl_c__cv_
                0x00000068                fldregobW_cv_
                0x00000030                bookmarK_cv_
                0x00000190                numtri2_cv_
                0x000001c4                __casl_funcs
                0x00000134                dpefF_cv_
                0x0000000c                invokersuB_cv_
                0x00000188                numtri1_cv_
                0x000001c4                grid_bindings
                0x0000005c                ide__pasS_cv_
                0x00000118                dpdiL_cv_
                0x00000178                numedC_cv_
                0x00000058                obpT_cv_
                0x0000004c                underlinE_cv_
                0x000001a8                numlmP_cv_
                0x00000170                numfroM_cv_
                0x00000160                numbishoP_cv_
 .data          0x00001358      0x980 casl_pilotmain.o
                0x000016bc                CASL_consts
                0x00001714                current_frame_menu
                0x0000173c                graffiti_indicator
                0x00001b9e                on_the_fly_object_id
                0x0000175e                white_pattern
                0x00001738                start_ticks
                0x00001720                pilot_pixel_ratio_y
                0x00001b7e                fontlist
                0x00001cce                system_colors_saved
                0x00001710                base_menu
                0x000016c0                num_const_bytes
                0x00001756                black_pattern
                0x0000174c                last_pen_x_frame
                0x0000135c                AppNetTimeout
                0x00001708                running_data_id
                0x0000135a                h_errno
                0x00001366                open_sockets
                0x00001cd4                casl_id
                0x00001730                msecs_per_tick
                0x00001358                AppNetRefnum
                0x00001ba2                physical_screen_y
                0x0000176c                biggest_chunk
                0x000016b8                this_object
                0x000016b6                num_objects
                0x000016c8                timer_root
                0x000016f4                basefont
                0x00001ba6                default_casl_app_info
                0x00001b76                fast_string_avail
                0x000016fc                casl_lib_handle
                0x00001cd0                using_color
                0x00001704                running_data_ref
                0x00001546                CASL_obj_properties
                0x00001740                hardware_buttons
                0x000016ee                screensize_y
                0x00001718                pilot_pixel_ratio_x
                0x0000173e                hardware_id
                0x0000172e                serial_port_id
                0x00001770                alloc_from_dyn_heap
                0x00001768                dynamic_free
                0x00001ba5                menu_cmd_bar_active
                0x0000136a                CASL_properties
                0x00001360                inetlibRefNum
                0x00001766                good_color_depth
                0x00001700                casl_lib_base
                0x000016c4                CASL_funcs
                0x000016f8                global_constant_index
                0x000016cc                current_category
                0x000016f0                caslsize_x
                0x00001ba0                physical_screen_x
                0x00001cd1                keyboard_launched
                0x00001cd2                sockets_used
                0x0000170c                base_form
                0x00001ba4                dont_fill_grid
                0x00001362                inetH
                0x00001750                last_pen_x_position
                0x000016b2                CASL_objects
                0x000016ce                current_category_string
                0x000016f2                caslsize_y
                0x00001776                fast_string
                0x0000172a                new_serial_mgr
                0x0000174e                last_pen_y_frame
                0x00001728                serial_lib
                0x000016ec                screensize_x
                0x00001772                min_dynamic_ram
                0x00001754                property_object_subscript
                0x00001752                last_pen_y_position
 .data          0x00001cd8       0x1c /prc-tools/H-i586-cygwin32/lib/gcc-lib/m68k-palmos/2.95.2-kgpd/libgcc.a(_floatex.o)
                0x00001cd8                _fpCCR
 *(.gcc_exc)

.bss            0x00001cf4      0x4e8
                0x00001cf4                bss_start=.
 *(.bss)
 .bss           0x00001cf4        0xc obwheel-sections.o
                0x00001cf8                __text__caslsupp
                0x00001cfc                __text__caslnetw
                0x00001cf4                __text__
 *(COMMON)
 COMMON         0x00001d00        0x2 obwheel.o
                0x00001d00                __casl_constants
 *fill*         0x00001d02        0x2
 COMMON         0x00001d04      0x4d4 casl_pilotmain.o
                0x00001d04                scratch_char_buf
                0x00001e94                color_depth
                0x00001e98                framergb
                0x00001e9c                errno
                0x00001ea0                platform_version
                0x00001ea4                fldhighliteforergb
                0x00001ea8                formbackrgb
                0x00001eac                forergb
                0x00001eb0                gNetLibOpen
                0x00001eb4                AppINETString
                0x00001ed4                cur_xpen
                0x00001ed8                text_fore_index
                0x00001edc                fldlinesrgb
                0x00001ee0                text_back_index
                0x00001ee4                AppServInfo
                0x00001f2c                selectedforergb
                0x00001f30                formforergb
                0x00001f34                AppHostInfo
                0x0000216c                fldhighlitebackrgb
                0x00002170                sock_objs
                0x00002184                frame_fore_index
                0x00002188                fldcaretrgb
                0x0000218c                frame_back_index
                0x00002190                backrgb
                0x00002194                selectedbackrgb
                0x00002198                generic_fore_index
                0x0000219c                object_ptr
                0x000021a0                inet_sock_objs
                0x000021c8                fldtextrgb
                0x000021cc                cur_ypen
                0x000021d0                generic_back_index
                0x000021d4                fldbackrgb
 COMMON         0x000021d8        0x4 netfile.o
                0x000021d8                linger_structure
                0x000021dc                end=ALIGN(0x4)
                0x000021dc                edata=ALIGN(0x4)
LOAD /prc-tools/H-i586-cygwin32/m68k-palmos/lib/gcrt0.o
LOAD obwheel.o
LOAD obwheel-sections.o
LOAD casl_pilotmain.o
LOAD caslprop.o
LOAD casl_events.o
LOAD casl_support_pilot.o
LOAD casl_support.o
LOAD netfile.o
LOAD pilotsock.o
LOAD casllib.a
LOAD obwheel-sections.ld

caslsupp        0x00000000     0x7328
 *(caslsupp)
 caslsupp       0x00000000     0x18a8 casl_events.o
                0x000016d4                _pda_objects_made
                0x000008f6                _pda_eventloop
                0x0000164e                _refresh_unbound_selected_grid_cells
                0x000016dc                _pda_objects_modified
 caslsupp       0x000018a8     0x37b2 casl_support_pilot.o
                0x00003fec                _pda_sdword_to_float
                0x00001ef6                _pda_any_dispose
                0x00003c70                _pda_exists
                0x00001fd4                _pda_randomn
                0x0000467c                _dbfile_rec_search
                0x00003ae6                _pda_set_color
                0x00003f6c                _pda_string_to_float
                0x00002102                _pda_clipboard
                0x00003cae                _pda_message_box
                0x000041bc                _pda_play
                0x00003238                _pda_close_file
                0x00003eee                _pda_set_category
                0x0000400c                _pda_byte_to_float
                0x00002286                _pda_bitmap
                0x00001e46                _pda_permanent_ptr
                0x000020b8                _pda_single_line
                0x0000475e                _pda_color_depth
                0x00001d14                _pda_malloc
                0x00001c72                _pda_new
                0x00003b36                _pda_last_pen_x
                0x00004702                _pda_rgb
                0x00004244                _pda_float_to_string
                0x00002a94                _pda_hide_object
                0x00002dbe                _pda_open_file
                0x00001e8c                _pda_any_memory
                0x00003ab6                _pda_elapsed_milliseconds
                0x00004020                _pda_boolean_to_float
                0x00004154                _pda_launch
                0x00003ede                _pda_get_category_string
                0x00003eca                _pda_get_category
                0x0000357a                _pda_rename_file
                0x00005032                _pda_get_dropdown_buffer
                0x00001d64                _pda_free
                0x00001dca                _pda_unlock_bitmap
                0x000033aa                _pda_remove_record
                0x00001b18                _pda_startup
                0x00003608                _pda_getfield
                0x00003fb8                _pda_float_to_sword
                0x00003514                _pda_delete_file
                0x0000216c                _pda_focus
                0x00004056                _pda_search_db
                0x00003f9e                _pda_float_to_word
                0x0000477e                _draw_grid_item
                0x0000232a                _pda_show_object
                0x00002046                _pda_list_exec
                0x00003fd2                _pda_float_to_sdword
                0x0000500e                _pda_put_dropdown_buffer
                0x000037b4                _pda_put_fields_or_insert
                0x00003b64                _pda_last_pen_y
                0x00001e06                _pda_dynamic_or_db_heap_alloc
                0x00003462                _pda_seek_file
                0x00001bda                _pda_globals_done
                0x00004044                _pda_userpath
                0x00001f66                _pda_write_mem
                0x000018a8                _pda_shutdown
                0x00001f9e                _pda_error
                0x00003b92                _pda_date_value
                0x00002010                _pda_attach_menubar_to_frame
                0x00001cae                _pda_dispose
                0x00003f1a                _pda_arm_timer
 *fill*         0x0000505a        0x2
 caslsupp       0x0000505c     0x22ca casl_support.o
                0x0000598c                _CASL_display_exec
                0x00005bbc                _CASL_shutdown
                0x00006582                _CASL_find
                0x000050e6                _CASL_attach_object_bitmap
                0x00006b6e                _CASL_select_object_list
                0x00005c64                _CASL_size_string
                0x00006b58                _CASL_select_object
                0x00005e04                _CASL_put_buffer
                0x0000505c                _CASL_attach_dbfile_fields
                0x000066f6                _CASL_mid
                0x000052b0                _CASL_property_str
                0x00006514                _CASL_abs
                0x00006c94                _CASL_string_make
                0x00006796                _CASL_right
                0x00005262                _CASL_property_num
                0x00005b4e                _CASL_geometry_exec
                0x000052fa                _CASL_startup
                0x00006dae                _CASL_strcmp
                0x000065f4                _CASL_trunc
                0x000068f2                _CASL_value
                0x00006b34                _CASL_run_function
                0x000067ea                _CASL_string
                0x00006682                _CASL_upper_lower
                0x00006d1a                _CASL_var_string_make
                0x00005e68                _CASL_put_generic
                0x000069a2                _CASL_add_to_draw_list
                0x00006dee                _CASL_strlen
                0x000060ba                _CASL_get
                0x00006bcc                _CASL_string_add
                0x000054e2                _CASL_apply_object_mods
                0x0000691c                _CASL_redraw_graphics
                0x00006490                _CASL_do_graphic_cmd
                0x00005cea                _CASL_put
                0x00006e36                _casl_fill_grid
                0x0000543c                _CASL_apply_global_mods
                0x000064e6                _CASL_asc
                0x000063ee                _CASL_move
                0x0000660e                _CASL_left
                0x0000655e                _CASL_char
                0x000051d2                _CASL_property_set
LOAD /prc-tools/H-i586-cygwin32/m68k-palmos/lib/libcrt.a
LOAD /prc-tools/H-i586-cygwin32/lib/gcc-lib/m68k-palmos/2.95.2-kgpd/libgcc.a
LOAD /prc-tools/H-i586-cygwin32/m68k-palmos/lib/libg.a
LOAD /prc-tools/H-i586-cygwin32/m68k-palmos/lib/libc.a
LOAD /prc-tools/H-i586-cygwin32/m68k-palmos/lib/libcrt.a
LOAD /prc-tools/H-i586-cygwin32/lib/gcc-lib/m68k-palmos/2.95.2-kgpd/libgcc.a
OUTPUT(obwheel coff-m68k)

caslnetw        0x00000000     0x76ec
 *(caslnetw)
 caslnetw       0x00000000     0x21f6 caslprop.o
                0x00001cb4                pda_property_bound_read
                0x00001628                pda_property_focused_object_read
                0x00000dd0                pda_property_number_of_records_read
                0x00001f52                pda_property_number_of_data_rows_write
                0x00001e04                pda_property_format_read
                0x00001f12                pda_property_number_of_data_rows_read
                0x0000088e                pda_property_display_write
                0x00000116                pda_property_width_write
                0x0000074e                pda_property_display_read
                0x0000130a                pda_property_checkbox_read
                0x00002092                pda_property_menubar_write
                0x0000048e                pda_property_x_position_read
                0x00001c74                pda_property_number_of_display_columns_read
                0x00000d66                pda_property_list_write
                0x00001c34                pda_property_number_of_display_rows_read
                0x000017ec                pda_property_foreground_read
                0x00000f08                pda_property_data_source_name_write
                0x00001006                pda_property_object_type_read
                0x000011a2                pda_property_list_size_write
                0x00001d92                pda_property_modified_write
                0x000009d2                pda_property_selected_write
                0x0000037e                pda_property_height_write
                0x000014f0                pda_property_focused_read
                0x000014b2                pda_property_cursor_write
                0x0000184a                pda_property_foreground_write
                0x000010cc                pda_property_no_input_write
                0x00001472                pda_property_cursor_read
                0x0000193a                pda_property_background_read
                0x00001700                pda_property_font_name_read
                0x00000f9e                pda_property_bitmap_write
                0x00001fb8                pda_property_menubar_read
                0x00000630                pda_property_y_position_write
                0x0000027c                pda_property_height_read
                0x00001aac                pda_property_object_string_write
                0x00001b6a                pda_property_bookmark_write
                0x00001a12                pda_property_object_string_read
                0x00001090                pda_property_no_input_read
                0x0000059e                pda_property_y_position_read
                0x00002196                pda_property_select_enable_write
                0x00000e48                pda_property_number_of_fields_read
                0x00000000                pda_property_width_read
                0x00001e78                pda_property_format_write
                0x00001996                pda_property_background_write
                0x00001232                pda_property_open_name_read
                0x00000d06                pda_property_hidden_write
                0x000004de                pda_property_x_position_write
                0x00000c28                pda_property_hidden_read
                0x00001360                pda_property_checkbox_write
                0x00000eaa                pda_property_data_source_name_read
                0x00002156                pda_property_select_enable_read
                0x000017c2                pda_property_font_name_write
                0x00001d24                pda_property_modified_read
                0x00001ed2                pda_property_old_bookmark_read
                0x00001160                pda_property_list_size_read
                0x00001b2e                pda_property_bookmark_read
                0x00001574                pda_property_focused_write
                0x00000970                pda_property_selected_read
 *fill*         0x000021f6        0x2
 caslnetw       0x000021f8     0x4b74 casl_support_pilot.o
                0x00006448                _serial_put
                0x000047b6                _pda_put_selector_num
                0x00004354                _pda_put_text_buffer
                0x0000603a                _set_graffiti_shift
                0x000021f8                _fixup_form_children
                0x000047ae                _pda_put_value_num
                0x0000463e                _pda_put_file_buffer
                0x00005816                _communications_open
                0x00005d86                _build_file_list
                0x000060e2                _network_get
                0x000045c0                _pda_put_filesel_buffer
                0x000031c0                _pda_scrollbar
                0x000061d0                _network_put
                0x00004bca                _pda_get_menuitem_buffer
                0x000064f8                _setup_color_draw
                0x0000620e                _serial_get
                0x00005012                _pda_get_value_num
                0x00004fda                _pda_get_filesel_buffer
                0x00003184                _pda_no_input
                0x000052da                _scroll_text
                0x0000501a                _get_float
                0x0000250a                _make_list_object
                0x000034e2                _pda_apply_geometry
                0x00005f08                _free_file_list
                0x000041bc                _pda_put_label_buffer
                0x00004d82                _pda_get_label_buffer
                0x00004cea                _pda_get_frame_buffer
                0x00004e12                _pda_get_text_buffer
                0x00004076                _pda_put_menuitem_buffer
                0x00004f98                _pda_get_selector_num
                0x000022ce                _make_base_menu
                0x00003f72                _pda_put_button_value
                0x00005ce0                _last_db_error
                0x000055b0                _init_form
                0x00004136                _pda_put_menutop_buffer
                0x00003d28                _pda_put_button_buffer
                0x00005456                _update_scroll_bar
                0x0000344c                _pda_border
                0x00004ffa                _pda_get_filesel_num
                0x000023e2                _layout_menu
                0x00004acc                _pda_get_button_buffer
                0x00002596                _pda_make_object
                0x00005d10                _get_app_info_id
                0x000058ca                _network_open
                0x00005a00                _serial_open
                0x00004ed0                _pda_get_selector_buffer
                0x00004172                _pda_put_frame_buffer
                0x0000569e                _init_scrollbar
                0x00005c84                _get_file_pointer
                0x0000483a                _pda_get_file_buffer
                0x00005f5c                _add_timer_rec
                0x0000681e                _cleanup_color_draw
                0x00003030                _pda_font
                0x00003922                _pda_position_object
                0x00005ff0                _get_non_deleted_record
                0x0000236c                _count_children
                0x0000257e                _make_resource_id
                0x00004c5a                _pda_get_menutop_buffer
                0x000068ec                _draw_frame
                0x0000527e                _get_parent_formptr
                0x00003a8e                _pda_graphic
                0x00003362                _pda_checkbox
 caslnetw       0x00006d6c      0x866 netfile.o
                0x0000735a                read_netfile
                0x0000754c                event_netfile
                0x00007132                close_netfile
                0x00006d86                open_netfile
                0x000071ec                write_netfile
 *fill*         0x000075d2        0x2
 caslnetw       0x000075d4      0x118 pilotsock.o
                0x000076a6                CloseNetwork
                0x0000763c                OpenNetwork
                0x000075d4                InitNetworkGlobals
                0x000075ec                FindNetworkLibrary

.reloc          0x00000000      0xa20
 .reloc         0x00000000      0x4e0 obwheel.o
 .reloc         0x000004e0      0x540 casl_pilotmain.o
